:1000000001308A005C29FF3FF30003088301EA0006
:100010000408EB000A08EC008A017408F100750876
:10002000F000030883120313E4000A08E3000C1E27
:10003000372883160C1E372883120317AC080319C0
:100040002E282B08103E8400831700080313990004
:100050001C300317AB0A2B020318AB01AC08031DBD
:100060003528831603130C123728AC03AC03831214
:1000700003138C1E8D2883168C1E8D288312981CCA
:100080004428181218168D28181D4B281A08831694
:10009000AF00831289280317EE0803195328403054
:1000A0006D02031C5728EF01ED01EE01EE0A6E0B05
:1000B0008828ED0A6D032D3E8400831703131A0868
:1000C00080000317EF0A6D082C3E84008317000898
:1000D0000313990003176D082C3E84008317000852
:1000E0000D3A031D7D280313061604308316A8005D
:1000F000023083120317EE008D286D082C3E840019
:1001000083170008083A031D8D28ED03ED038D28A1
:1001100003131A089A001A089A008B1C96288B1051
:1001200083120313061604308316A80083120313E8
:100130008C1C4B298316A8080319A228A80BA228F7
:10014000831206128316A3080319AA28A30BAA2850
:1001500083120611633083162C020318FA28AC0AA6
:10016000003037022E3003193602A01CCB28031CA6
:10017000C728033037025230031936020318C52846
:100180000A30B6070318B70ADC28A010DC28B60A24
:100190000319B70ADC28031CCF28F630D728003013
:1001A0003702023003193602031CDB28FF30B60782
:1001B000031CB703DC28A0143708F5003608F40048
:1001C0000310F50CF40C0310F50CF40C74088312F6
:1001D0009B008316B61CEF2883129D16F12883120C
:1001E0009D128316361CF72883121D164829831288
:1001F0001D124829831210100F08E6000E08E500B2
:100200006608F5006508F40083163808F402031C3C
:10021000F5033908F502750874040319172927082E
:10022000D13E840083133808831265021F292708F2
:10023000D13E840083138312650883163802800040
:100240008316390883126606031D2A298316380887
:1002500083126506031D322983162708D13E8400C8
:1002600083138001831265088316B8008312660821
:100270008316B900831210148316A70A27080A3AB6
:100280000319A7010A302B02031CAB0AAC0120158D
:10029000831285128C1063088A0064088300710839
:1002A000F4007008F5006B0884006C088A006A0886
:1002B0008300F30E730E09006F1083196F14EF1093
:1002C000031AEF142030840067307921A0308400B5
:1002D000EA30792183171030840070307921831639
:1002E0000317900183010A168A11492B0406800125
:1002F000840A0406031D7629640000348312031364
:10030000ED00EE1B8C296E1B94296E088A006D0887
:10031000ED0A0319EE0A820083136E1883176D0825
:10032000ED0A8400000808000A340D3445344534D1
:10033000503452344F344D342034443441344334F7
:100340005F3450346C347534733420344834693439
:10035000673468343D3420342534753400340A342D
:100360000D344E346534773420344E3420347634B2
:1003700061346C34753465343D342034253475343F
:1003800000340A340D3445344534503452344F343B
:100390004D3420344E342034563461346C3475344A
:1003A00065343D3420342534753400340A340D343A
:1003B0004E346534773420344434413443345F342C
:1003C00050346C34753473342034483469346734B1
:1003D00068342034433461346C34693462347234A8
:1003E0006134743469346F346E3420343D342034D5
:1003F0002534753400340A340D3443347534723482
:10040000723465346E3474342034443441344334AB
:100410005F3450346C347534733420344834693468
:10042000673468342034433461346C346934623462
:1004300072346134743469346F346E3420343D3432
:1004400020342534753400340A340D344334753483
:100450007234723465346E34743420344E34203443
:10046000763461346C347534653420343D34203452
:100470002534753400340A340D3457345334203461
:10048000203420343D3420345734613472346D3498
:1004900020345334743461347234743400340A3484
:1004A0000D34453444344634203420343D34203433
:1004B0007734723469347434653420346434653488
:1004C0006634613475346C347434203445344534C6
:1004D000503452344F344D342034763461346C34DB
:1004E00075346534733400340A340D344D3461345A
:1004F00078342034773469346E346434203473347F
:10050000703465346534643420343D34203425340B
:1005100035342E343234663420346D342F34733411
:1005200000340A340D343134303420346D346934BD
:100530006E342E3441347634653472346134673429
:1005400065342034573469346E3464342034533481
:10055000703465346534643420343D3420342534BB
:1005600035342E343234663420346D342F347334C1
:1005700000340A340D344634613473347434203416
:10058000573469346E3464342034533470346534F1
:100590006534643420343D342034253464342034CC
:1005A0006D342F34733400340A340D3445344534FB
:1005B000503452344F344D34203453346534723413
:1005C000693461346C3420344E3475346D346234A3
:1005D000653472343D34203423342534733400348C
:1005E0000A340D3455346E34693474342034533441
:1005F00065347234693461346C3420344E3475346B
:100600006D34623465347234203420342034203424
:10061000203420342034203420342034203420343A
:1006200020343D34203423342534733400340A34E8
:100630000D342534733420342534733400340A34B3
:100640000D34433456345334203420342034203491
:100650002034203420343A342034253473340034A8
:100660000A340D342534733400340A340D345234D2
:1006700046342034203420343D342034533465341F
:100680007434203452346F3474346F347234203400
:1006900046346134633474346F34723400340A3451
:1006A0000D34523446345334203420343D34203415
:1006B000533474346F3472346534203452346F34AC
:1006C00074346F3472342034463461346334743497
:1006D0006F34723400340A34413454343F3420349B
:1006E00066346F3472342034683465346C3470345A
:1006F00000340A340D34493420342034203420347A
:100700003D342034763465347234733469346F3454
:100710006E34203469346E3466346F3400346F3490
:100720006B3400340A340D34443450344834533478
:1007300020343D342034533474346F34723465348F
:100740002034443441344334203450346C347534D0
:1007500073342034483469346734683400340A34DC
:100760000D34443450344834203420343D34203463
:10077000443441344334203450346C34753473344D
:1007800020344834693467346834003420342834E1
:1007900063342934203432343034303437342D3417
:1007A000323430343034383420344B344F344334E2
:1007B0004834203445346E34673469346E346534DB
:1007C0006534723469346E34673400340A340D345D
:1007D00052346F346C346C3469346E346734413461
:1007E0007634653472346134673465345334753427
:1007F0006D3420343D342034253435342E343234B5
:10080000663400340A340D34253435342E34323411
:10081000663400340A340D344E3465347734203471
:1008200052346F3474346F3472342034463461344B
:10083000633474346F3472343D3420342534663478
:1008400000340A340D3443347534723472346534F0
:100850006E347434203452346F3474346F347234E0
:10086000203446346134633474346F3472343D342C
:1008700020342534663400340A340D34453445348C
:10088000503452344F344D34203452346F34743435
:100890006F347234203446346134633474346F34CA
:1008A00072343D3420342534663400340A340D3437
:1008B00058344E342034203420343D3420347334C2
:1008C00065347434203441347634653472346134A0
:1008D000673469346E34673420344E342D345634E2
:1008E00061346C347534653400340A340D346D343D
:1008F000613478345B34253464345D3420346334BB
:100900006F3475346E3474343D342534643420349B
:100910006134673465343D342534643400340A343A
:100920000D344E346F344F3466344234753466348B
:10093000663465347234313430346D3469346E3435
:10094000563461346C3475346534733420343D343A
:1009500020342534643400340A340D346C3461346A
:10096000733474345F3463346F3475346E34743478
:1009700065347234763461346C34753465342034C3
:100980003D3420342534643400340A340D34733457
:1009900075346D3420346F34663420346C346134F3
:1009A00073347434203433342034763461346C340A
:1009B00075346534733420346F34663420346234D3
:1009C000753466346634653472345F34313473346C
:1009D000653463345B3469346E346434653478343C
:1009E0005D3420343D3420342534643400340A34FA
:1009F0000D34733475346D3420346F3466342034E0
:100A00006234753466346634653472345F3431343C
:100A10007334653463345B3430342E342E343934DB
:100A20005D3420343D3420342534643400340A34B9
:100A30000D346234753466346634653472345F3430
:100A400031347334653463345B34253464345D3459
:100A500020343D3420342034203420342534643490
:100A600000340A340D3425346434003425346334BE
:100A700000343C342D342D344E3445345734003456
:100A8000573469346E346434533465346E3473349B
:100A90006F347234203454347934703465342034F3
:100AA0004B344534323430344134533400340D3413
:100AB0004534523452344F34523400340A340D34F5
:100AC0002E342E342E3464346534663461347534F7
:100AD0006C3474342034763461346C347534653459
:100AE0007334203477347234693474347434653434
:100AF0006E34203474346F342034453445345034EB
:100B000052344F344D3400340A340D344634613499
:100B1000733474342034573469346E34643420347C
:100B200053347034653465346434203441346C3467
:100B3000613472346D342034543472346534733417
:100B400068346F346C34643420343D3420342534BC
:100B5000643420346D342F3473340A340A340D3441
:100B60003E3400340A340D347334613476346934DD
:100B70006E346734203474346F3420344534453453
:100B8000503452344F344D342E342E342E340034FD
:100B9000203420342A342A342A3420345734493437
:100BA0004E34443453345034453445344434203482
:100BB00041344C34413452344D3420342A342A34B4
:100BC0002A3400340A340D346C3461347334743490
:100BD0002034313420347334653463342E3420347B
:100BE000703475346C3473346534203463346F344A
:100BF00075346E34743420343D34203400340A3477
:100C00000D346E346F347734203472346534733479
:100C100065347434743469346E3467342E342E344D
:100C20002E340A340D3400340A340D342E342E346C
:100C30002E340A340A340D3400340008F400840AD7
:100C40000008F500840A0008F600840A0008F7008E
:100C5000212F83120313E901760D770DE700670852
:100C60000319362EE90DF701F6170800F401F50116
:100C7000F601F7010034E9107A0D7B0DE8006808F1
:100C80000319472E0318E914FB01FA170800E801BD
:100C9000F801F901FA01FB01080067080319362E73
:100CA000F613E90C670CF7000318F6174E2FE70848
:100CB00003197D2E770803196D2E77030319F40AA3
:100CC0000319F50A0319F60A0319F70A0310F70CBA
:100CD000F60CF50CF40CE70A572E7408750476042C
:100CE000770403197D2EF61B4D2EE70303197D2E85
:100CF0000310F40DF50DF60D732EF401F501F60158
:100D0000F7014E2F750D760D00380319080080305D
:100D1000F60608000310FF30F407F409031CF5077A
:100D2000F509031CF607F609031CF707F709080085
:100D3000840183120313E701FC01FD01FE01FF01A1
:100D4000780879047A047B040319A92EC030E705DA
:100D5000B42EF401F501F601F7014E2F0310F80D42
:100D6000F90DFA0DFB0DE70AFB1FAE2EE70A031083
:100D7000FC0DFD0DFE0DFF0D7B087702031DCA2E35
:100D80007A087602031DCA2E79087502031DCA2E41
:100D900078087402031CDC2E7C147808F4027908AD
:100DA000031C790FF5027A08031C7A0FF6027B0800
:100DB000031C7B0FF7020310FB0CFA0CF90CF80C68
:100DC000E70367083F39031DB72E671FF42E031092
:100DD000FF30F407F409031CF507F509031CF607B7
:100DE000F609031CF707F7097408F8007508F900FD
:100DF0007608FA007708FB007C08F4007D08F5000F
:100E00007E08F6007F08F700E71F4E2F0310FF3023
:100E1000F407F409031CF507F509031CF607F609A6
:100E2000031CF707F7094E2F0008F400840A000896
:100E3000F500840A0008F600840A0008F700992EDD
:100E400084017408FC007508FD007608FE00770830
:100E5000FF00F601F701F401F5010310FF0CFE0C91
:100E6000FD0CFC0C031C422F7808F40779080318CA
:100E7000790FF5077A0803187A0FF6077B0803182D
:100E80007B0FF7077C087D047E047F0403194E2F37
:100E90000310F80DF90DFA0DFB0D2D2F8408031921
:100EA0000034770880008403760880008403750886
:100EB00080008403740880000034F400F8010310FB
:100EC000FD307507031C842FF701F0307505031DF5
:100ED0006C2F0430F700F50EF6010310F70AF50D3C
:100EE000031C6E2FF50C750874020318F400F60D40
:100EF000F70B722FF81F7E2FF609F60A7608F81FF7
:100F00000800F409F40A0800F50C03188D2FF50CFD
:100F1000031CF4010310F40C031C03107408F60006
:100F2000F401F40D7A2FFA01F801F901760877043B
:100F3000031D9D2FF401F50100341F30FA04031046
:100F4000FA0AF60DF70D031CA02FF70CF60C770824
:100F50007502031DAD2F76087402031CB52F7608A9
:100F6000F4027708031C770AF502F80DF90DFA0B65
:100F7000FA1AA52FFA1FC12FF809F80A0319F90365
:100F8000F9097808F6007908F7007A1F0034F409A7
:100F9000F40A0319F503F509003483013008AF00A2
:100FA000D82FAF033F30A0000000A00BD42F640067
:100FB00001302F020318D12F2F08B0000310B00CFE
:100FC0000310300CA0000000A00BE32F0800F82F46
:100FD0006400981CF12F8316981298168312181229
:100FE0001816181DF82F1A08A100831698129816C3
:100FF000831203138C1EE82F1A08080083010034A3
:10100000FF3FFF3FFF3FFF3F00300A168A15DE2AF1
:1010100004308301AF003E30A0000000A00B0D287B
:101020006400AF0B0B28FF30AF07031CB003300880
:101030002F04031908000828F801F9010310F70C20
:10104000F60C031C2A287408F80775080318750A9B
:10105000F9070310F40DF50D760877040319003431
:101060001E2802308301AF00B0013630B1003108D4
:101070000038031944286400B0080319B103B00311
:101080008C1E37281A080800AF0B3428003483015F
:10109000C901CA01CB01CC0148084704031DBA2885
:1010A000F401F501F601F70108004808EE004708D1
:1010B0000A128A117E210A128A15CD0030304D02A3
:1010C000031C6F284808EE0047080A128A117E2187
:1010D0000A128A15CE003A304E02031C7428F4011D
:1010E000F501F601F70108000A30F800F901FA01EC
:1010F000FB014908F4004A08F5004B08F6004C08CB
:10110000F7000A128A1120274808EE0047080A1241
:101110008A117E210A128A15CD00CE01D030CD076A
:101120000318CE0AFF30CE074D08F8004E08F9002C
:10113000FA01FB0174087807FC007908FD007508C6
:101140000318750FFD077A08FE0076080318760F5E
:10115000FE077B08FF0077080318770FFF077C085E
:10116000C9007D08CA007E08CB007F08CC00C70AF2
:101170000319C80A4808EE0047080A128A117E219E
:101180000A128A150038031D55284908F4004A0838
:10119000F5004B08F6004C08F70008008301CF006B
:1011A00003178D0003134E0803178C0083168C134E
:1011B000031320108B1B201403170C158B135530B1
:1011C0008D00AA308D008C14831203130D1EE428A9
:1011D0000D12831603170C110313201CF1288B1713
:1011E000F2288B13831208008301CD004B08CE0038
:1011F0004D08CE204C08CE004D0ACE288301C900F0
:10120000CA0113294708840083130008CB00CC01CE
:101210004908F42008300A168A112E230A128A156A
:10122000C90AC70ACA0A48084A020318080002295C
:101230008301C70061304702031C24297B30470229
:1012400003182429E030C707470808008312031752
:101250006E08023A031D632E0330EE002D0818219C
:10126000413A031D292E03172E081821543A8316DC
:10127000031D2A2EA1018312061504308316A30034
:10128000831203172F08493A03194A292F08693A8C
:10129000031D5B2930300313C8000330C90001303F
:1012A000C1001030C2004130C7000A128A15042064
:1012B0000A128A152C2E2F0818214C3A0317031DE9
:1012C0006A2930081821303A031D69298316A501BF
:1012D0002C2E03172F0818214C3A0317031D7A29C7
:1012E00030081821313A031D79298316A501A50A72
:1012F0002C2E03172F0818214C3A0317031D8A2997
:1013000030081821323A031D892902308316A500BE
:101310002C2E03172F0818214C3A0317031DBB2945
:1013200030081821433A031DBA298316A601053057
:10133000260203182C2E0330F50026080A168A15FB
:101340000F21DB3E8400831380010330F500260863
:101350000A168A150F210A128A1503138312C30075
:10136000430ADB3E840083138001840A80018316D4
:10137000A60A972903172F081821453A0317031DBA
:10138000002A30081821443A0317031D002A3108A7
:101390001821463A031DFF2958308316BA0002303F
:1013A000BB00BA308312BB00C7000230C800403017
:1013B000FE200E308316C6008F30C7003F30C800B5
:1013C000C6308312BB00C7000330C8001030FE20B7
:1013D000C0308316B2000D30B300B2308312BB00B0
:1013E000C7000230C8002030FE205E30C800053043
:1013F000C9000A128A1504200A128A152C2E031716
:101400002F081821583A0317031D9B2A300818216A
:101410004E3A0317031D9B2A310818213D3A031742
:10142000031D9B2A32080D3A0319E22D32083F3A78
:10143000031D2F2A24300313C8000230C90083166D
:101440003A088312C10083163B088312C200413060
:10145000C7000A128A1504200A128A152C2E05309C
:1014600083160313A600831203176F080313C30028
:10147000C401FF30C307031CC40783162608831268
:10148000C500C6014608803AF4004408803A740258
:10149000031D4C2A43084502831626080318762AA2
:1014A0002D3E8400831700088312C300831626088C
:1014B000FB3E253E840083138312430880003630B0
:1014C000C8000530C90083162608FB3E253E84006F
:1014D00000088312C100C2014130C7000A128A15F8
:1014E00004200A128A158316A60A332AFB3E253EDB
:1014F00084008313800125308312C7008030C80028
:10150000472074088316BA007508BB00AF308312F9
:10151000C8000130C90083163A088312C10083163F
:101520003B088312C2004130C7000A128A1504200A
:101530000A128A152C2E2F081821583A0317031D5A
:10154000E02A300818214E3A0317031DE02A31081B
:101550001821533A031DDF2AB230C8000530C900F4
:101560000A128A1504200A128A15BA30BB00C70075
:101570000230C8004030FE208F30C8000330C90060
:101580000A128A1504203B08C7000230C800403008
:101590000A168A113E22C130C8000130C9008316E4
:1015A0003A088312C10083163B088312C2004130FF
:1015B000C7000A128A1504200A128A152C2E031756
:1015C0002F081821573A0317031DF62A300818214F
:1015D000533A031DF52AFF30C8000530C9000A122E
:1015E0008A1504200A128A11002803172F081821CF
:1015F000523A0317031DBC2B30081821463A031733
:10160000031DBC2B310818213D3A0317031DBC2BC9
:1016100032080D3A0319E22D32083F3A031D292BF7
:1016200021300313C8000430C90083164608831212
:10163000C000831647088312C1008316480883122E
:10164000C2004030C7000A128A1504200A128A1507
:101650002C2E053083160313A600831203176F0880
:101660000313C300C401FF30C307031CC407831660
:1016700026088312C500C6014608803AF4004408D3
:10168000803A7402031D462B430845028316260840
:101690000318702B2D3E8400831700088312C300AB
:1016A00083162608FB3E253E8400831383124308DD
:1016B00080003630C8000530C90083162608FB3E7E
:1016C000253E840000088312C100C2014130C700DA
:1016D0000A128A1504200A128A158316A60A2D2BCF
:1016E000FB3E253E84008313800125308312C70012
:1016F0008030C80047207408BC007508BD0076081B
:10170000BE007708BF003E043D043C040319A32B30
:101710003C08F4003D08F5003E08F6003F08F700DD
:101720000A128A15E427B730F700D130F8003830B4
:10173000F9000A128A15802774088316C6007508F6
:10174000C7007608C8000A308312C8000430C900F8
:10175000831646088312C000831647088312C1000F
:10176000831648088312C2004030C7000A128A1547
:1017700004200A128A152C2E2F081821523A03171A
:10178000031D062C30081821463A0317031D062CAA
:1017900031081821533A031D052CB230C80005301A
:1017A000C9000A128A1504200A128A15C630BB0025
:1017B000C7000330C8001030FE208F30C80003304F
:1017C000C9000A128A150420C630BB00C7000330C6
:1017D000C80010300A168A113E223C30C80004307E
:1017E000C900831646088312C00083164708831277
:1017F000C100831648088312C2004030C7000A1295
:101800008A1504200A128A152C2E03172F08182176
:10181000443A0317031D932C30081821503A03173C
:10182000031D932C31081821483A0317031D932CEC
:10183000320818213D3A0317031D932C33080D3A43
:101840000319E22D33083F3A031D3B2CFB300313F1
:10185000C8000130C900831632088312C100831604
:1018600033088312C2004130C7000A128A150420CF
:101870000A128A152C2E063083160313A600831233
:1018800003176F080313C300C401FF30C307031C11
:10189000C407831626088312C500C6014608803A8D
:1018A000F4004408803A7402031D582C4308450292
:1018B0008316260803186E2C2D3E8400831700081B
:1018C0008312C30083162608FA3E253E8400831344
:1018D0008312430880008316A60A3F2CFA3E253E59
:1018E00084008313800125308312C7008030C80034
:1018F000472074088316B2007508B300D6308312EF
:10190000C8000130C900831632088312C100831653
:1019100033088312C2004130C7000A128A1504201E
:101920000A128A152C2E2F081821443A0317031D7A
:10193000DF2C30081821503A0317031DDF2C310823
:101940001821483A0317031DDF2C32081821533A97
:10195000031DDE2CB230C8000530C9000A128A15FA
:1019600004200A128A15B230BB00C7000230C8003A
:101970002030FE208F30C8000330C9000A128A15BB
:101980000420B230BB00C7000230C80020300A1665
:101990008A113E229430C8000130C90083163208F3
:1019A0008312C100831633088312C2004130C7007E
:1019B0000A128A1504200A128A152C2E03172F08E2
:1019C0001821443A0317031DFB2C30081821313A23
:1019D000031DFA2C3130C8000530C9002308C100AE
:1019E0002408C2004130C7000A128A1504200A12D6
:1019F0008A152C2E03172F081821443A0317031DAC
:101A00002A2D30081821323A031D292D0230C80032
:101A10000430C90083164608F7004708F800480854
:101A2000F9004008F4004108F5004208F6000A12E7
:101A30008A15802774088312C0007508C1007608D3
:101A4000C2004030C7000A128A1504200A128A1503
:101A50002C2E03172F081821443A0317031D5F2D5E
:101A600030081821333A031D5E2D0230C8000430BF
:101A7000C90083165B08F4000A128A157A26F7015A
:101A80004030F800F9000A128A153F274608F7008F
:101A90004708F8004808F9000A128A1580277408D8
:101AA0008312C0007508C1007608C2004030C7002C
:101AB0000A128A1504200A128A152C2E03172F08E1
:101AC0001821533A0317031DE52D300818214E3A0B
:101AD0000317031DE52D310818214E3A0317031D86
:101AE000E52D32083D3A031DE22D3308213A031D4E
:101AF000E22DB2300313C8000530C9000A128A155E
:101B000004200A128A1507308316A60083120317D1
:101B10006F080313C300C401FF30C307031CC407CD
:101B2000831626088312C500C6014608803AF400D1
:101B30004408803A7402031D9F2D43084502831612
:101B400026080318B52D2D3E840083170008831244
:101B5000C30083162608F93E253E840083138312B2
:101B6000430880008316A60A862DF93E253E840090
:101B70008313800125308312BB00C7000A30C800E0
:101B80000030FE208F30C8000330C9000A128A15C9
:101B90000420CC30BB00C7000A30C80000300A1651
:101BA0008A113E22D430C8000230C900CC30C100B6
:101BB0008030C2004130C7000A128A1504200A1280
:101BC0008A152C2E831603132A2E2F0818213F3A2C
:101BD000031D252EAF30C8000330C9000A128A1534
:101BE00004209230C8000330C9000A128A1504206C
:101BF0004F30C8000230C9000A128A15042079301B
:101C0000C8000330C9000A128A1504203530C80004
:101C10000330C9000A128A1504204F30C80003306F
:101C2000C9000A128A1504203B30C8000230C900DE
:101C30000A128A1504205630C8000430C9000A125E
:101C40008A1504200A128A152C2E03308316A1004F
:101C50002C2E8316A101A10A8316210B302E342EBF
:101C60002108033A031D432E57308312C800053064
:101C7000C9000A128A1504206B30C8000330C9005D
:101C80000A128A150420AE308312C8000530C9003C
:101C90000A128A1504200A128A158316AF018312CC
:101CA00003176F08831603132F020318592EAF0A68
:101CB0004F2E2F082D3E84008317800183120317B7
:101CC000ED01EF01EE01031308008408031900344D
:101CD00076088000840375088000840374088000FF
:101CE0000034F501F601F701F41FE92FF503F603BF
:101CF000F703E42FF501F601F701E92FFC01750D5B
:101D0000760DFA007A080319892EFC0DF601F517F5
:101D10000800F401F501F6010034FC10780D790D8E
:101D2000FB007B080319992E0318FC14F901F8171E
:101D30000800FB01F701F801F90108007A0803190E
:101D4000892EF513FC0C7A0CF6000318F517652E96
:101D5000FA08031DBC2EF401F501F601652E760389
:101D60000319F40A0319F50A0319F60A0310F60C0D
:101D7000F50CF40CFA0AA82EF608031DAF2E740811
:101D800075040319AB2EF51B9E2EFA030319AB2E17
:101D90000310F40DF50DC32E8030F9060008F40091
:101DA000840A0008F500840A0008F600F22E7A087A
:101DB0007B02031CE62E031908000310F60CF50C39
:101DC000F40CFA0A7A087B02DB2E0310F90CF80CEB
:101DD000F70CFB0A7A087B0603190800E52E803011
:101DE000F90684017E268D26D7267C1CFF2EF40959
:101DF000F509F609F40A0319F50A0319F60AFC1C99
:101E0000092FF709F809F909F70A0319F80A03195C
:101E1000F90A7708F40778080318780FF5077908A6
:101E20000318790FF607FC01F61FA82EF409F5092F
:101E3000F609F40A0319F50A0319F60A7C14A82E08
:101E40007608790680390319292F790D7908013828
:101E50000800F61379087F397602031D372F7808BA
:101E60007502031D372F7708740203190800030851
:101E70000238F91B013A83000318803808008401F6
:101E80007E268D26FD01FE01FF01FA0803190800D8
:101E90007B08031908007A02773EFA007C0CFC06E6
:101EA0001830F9000310FD0DFE0DFF0D7608031D1F
:101EB000612F78087502031D5F2F77087402031CD9
:101EC0006B2F7708F4027808031C780FF502031CC7
:101ED000F6037D140310F40DF50DF60DF90B522FDA
:101EE0007D08F4007E08F5007F08F600A82E0008A3
:101EF000F400840A0008F500840A0008F600812F27
:101F000084017E268D26FD01FE01FF010730F900C8
:101F10000310F80CF70C031C982F7408FD077508C4
:101F20000318750FFE0776080318760FFF070310D6
:101F3000F40DF50DF60DF90B882F0930F900A42FDB
:101F40000310FF0CFE0CFD0C0310F80CF70C031C27
:101F5000B32F7408FD0775080318750FFE07760880
:101F60000318760FFF07F90BA02F7C0CFC067D08E9
:101F7000F4007E08F5007F08F6007A307B07FA0748
:101F8000A82E84017E26F7018230FA07FA1B892EDB
:101F9000F030FA07FA1BDD2F18307A020318892E69
:101FA000FA08031DD62F7C188A260800FA030310AE
:101FB000F40DF50DF60DF70DD02F0310F60CF50C02
:101FC000F40CFA0FDD2FD32FF71FE92F7C148A268C
:101FD000EA2FFC018E30FA008401F7080319A82EBD
:101FE0000310F70CF60CF50CF40CFA0AED2FF601C1
:101FF000F51BF6037608F700E42FF601F701E92F49
:102000008207243452346534763469347334693445
:102010006F346E343A34203431342E343234303428
:10202000203424340034FF3FFF3FFF3FFF3FFF3F9A
:10203000FF3F8301AF000430B0003E30A00000003D
:10204000A00B1F28B00B1D28AF0B1B280800830115
:10205000981C302883169812981683121812181696
:10206000181D37281A08A100831698129816831293
:1020700008008301BB013B0ABC0005303C02031889
:1020800067290330F5003B080A168A150F21DB3E4D
:10209000840083130008BD000330F5003C080A16D5
:1020A0008A150F210A168A11DB3E8400831300086B
:1020B0003D020330F5000318D4283B080A168A15A0
:1020C0000F21DB3E8400831300088316C900033010
:1020D000F50083123B080A168A150F21BD003D0A40
:1020E000DB3E8400831300088316CA00840A0008BC
:1020F000CB000330F50083123C080A168A150F2125
:10210000DB3E840083130008BD000330F5003B086C
:102110000A168A150F21DB3E840083133D088000D8
:102120000330F5003C080A168A150F21BD003D0A50
:10213000DB3E840083130008F400840A0008F500E5
:102140007408BE007508BF000330F5003B080A168E
:102150008A150F21C000400ADB3E840083133E082D
:102160008000840A3F0880000330F5003C080A160E
:102170008A150F21DB3E84008313831649088000F3
:102180000330F50083123C080A168A150F21BD00A2
:102190003D0ADB3E8400831383164A088000840ACC
:1021A0004B0880000330F50083123B080A168A159D
:1021B0000F21DB3E840083130008BD000330F500CF
:1021C0003C080A168A150F210A168A11DB3E840084
:1021D000831300083D06031D64290330F5003B0806
:1021E0000A168A150F21BD003D0ADB3E84008313C9
:1021F0000008F400840A0008F5007408BE007508A1
:10220000BF000330F5003C080A168A150F210A1694
:102210008A11C000400ADB3E840083130008F400EA
:10222000840A0008F5003F087502031D19293E08BD
:102230007402031864290330F5003B080A168A1556
:102240000F21BD003D0ADB3E840083130008831686
:10225000CA00840A0008CB000330F50083123C0852
:102260000A168A150F21BD003D0ADB3E8400831348
:102270000008F400840A0008F5007408BE00750820
:10228000BF000330F5003B080A168A150F21C00075
:10229000400ADB3E840083133E088000840A3F0826
:1022A00080000330F5003C080A168A150F210A1633
:1022B0008A11BD003D0ADB3E8400831383164A0861
:1022C0008000840A4B0880008312BC0A3D28BB0AA8
:1022D00005303B02031808003B2883014108F50044
:1022E0004008F4000A128A15FD27F7018030F80033
:1022F0003F30F9000A128A15F1267408F7007508B4
:10230000F8007608F900F401F5014030F6000A12F1
:102310008A153F277408C5007508C6007608C700EF
:102320004508F7004608F8004708F900F401803036
:10233000F5003F30F6000A128A15EF263D08F70037
:102340003E08F8003F08F9000A128A158027740831
:10235000C8007508C9007608CA003C08F5003B08AB
:10236000F4000A128A15FD274508F7004608F80010
:102370004708F9000A128A1580274808F70049081B
:10238000F8004A08F9000A128A15F1260A168A117D
:102390007408C2007508C3007608C4004208F4003F
:1023A0004308F5004408F6000800831603132508C7
:1023B000023A031D222AA6010A3026020318222A05
:1023C00017308312C8000530C90083162608D13E95
:1023D0008400831300088312BD00BE018316260803
:1023E0008312BB00BC013B30C7000A128A150420CF
:1023F0000A168A110930831626020318122A2608A3
:102400008312BF00C0010130BF070318C00A831642
:10241000270883123F064004031D1F2A3930C800D5
:102420000530192AA708031D1F2A39308312C80056
:102430000530C9000A128A1504200A168A1183166B
:10244000A60ADC29831208008301CE0003178D0041
:1024500083168C130C1483120C08031308008301D9
:10246000CB004B0A2422CD00CC014B082422F400DF
:10247000F5014C08F4044D08F50408008301C90077
:10248000CA014F2A47088400831349082F220A16DD
:102490008A11740883138000C90AC70ACA0A480847
:1024A0004A0203180800422A8301BF00C101BF0885
:1024B000031D5C2A3F0B5E2AC101C10ABB08031D34
:1024C000632A3B0B652AC101C10ABC08031D6A2AA5
:1024D0003C0B6C2AC101C10A10303E0200300319C6
:1024E0003D02031C752AC101C10A071287123F0C65
:1024F000031C7C2A87157D2A8711071607120716E9
:1025000007123B0C031C862A8715872A871107169A
:1025100007123C0C031C8E2A87158F2A8711071679
:10252000071210303E02003003193D02031C9C2AA2
:10253000FF30BD000F30BE00BD0EBE0EF030BE0538
:102540003D080F39BE04F030BD05C001C00A0310BC
:10255000BD0DBE0D031CAE2A8715AF2A871183124D
:10256000031307160712C00A0D304002031CA82AE5
:102570008716410808008301BB01BB0ABC01BC0AE5
:1025800083164308F7004408F8004508F9000030B6
:10259000F401F501F6010A128A158027F701F80106
:1025A0003F30F9000A128A15F1260A128A15C1274E
:1025B0000A168A1174088312BD007508BE00013026
:1025C00054228316A2008312BB01BC01BC0A8316ED
:1025D0003308F5003208F4000A128A15FD27F701C6
:1025E000F030F8004130F9000A128A153F274308FD
:1025F000F7004408F8004508F9000A128A158027F8
:10260000F701F8013F30F9000A128A15F1260A1283
:102610008A15C1270A168A1174088312BD0075082D
:10262000BE00003054228316A20083120711071542
:1026300008000B3083160313990018151812831223
:1026400098171816981283160C128C1218138312EE
:102650001813831698129816831208008301CB0072
:102660000430CC003E30A0000000A00B342B6400EE
:10267000CC0B322BCB0B302B08008301AF00043086
:10268000B000FA302E236400B00B412BAF0B3F2B70
:1026900008000F3083160313850001308600813057
:1026A00087008B13831206110612871006156430FB
:1026B0002E2306116400061664302E2306126400D1
:1026C000871464302E238710FF3083168100640046
:1026D00019238316B601B60AB701A010A401A501FB
:1026E00083121F1083169F111F159F149D131D1316
:1026F000831210108F018E01971117159710171460
:102700009014901190121012101183160C10831255
:102710001014921412108F30831692008312121329
:10272000921212169215121583168C1401130B16A1
:1027300064000B178B128B110D120C138C120C12E0
:102740008C110C110D108D110D13A701AD2B270845
:10275000D13E840083138001A70A0A302702031C9C
:10276000A72BA7010C108C1483120F088316B90035
:1027700083120E088316B8008312061206158614FB
:102780009D151D159501640005080F398316AD00D0
:102790008312BB01BB0ABC01BC0ABD011030BE00E4
:1027A000003054228316A2008312BB01BB0ABC0175
:1027B000BC0ABD01BE01013054228316A20083125F
:1027C0000711071583168C16072CAE01AE0A282CAC
:1027D0000230032C0330032C0430032C0530032C6F
:1027E0000630032C0730032C0830032C0930032C4F
:1027F0000A30032C0B30032C0C30032C0D30032C2F
:102800000E30032C0F30AE00282CAE01282C2D08E2
:10281000F400F03E0318052C103E031C052C00307C
:10282000F40214308A001830740703188A0A8200F0
:10283000282CE52BE82BEA2BEC2BEE2BF02BF22BA4
:10284000F42BF62BF82BFA2BFC2BFE2B002C022C56
:10285000640017308312C8000330C900C630B600C8
:102860000330B7004030B4000530B5003430C70045
:102870000A128A1504201F30C8000330C900013035
:10288000B6001030B7003630C7000A128A1504208F
:102890000A168A11CC30A200C7000A30C8000030E6
:1028A0003E22F030C8000230C900CC30B600803083
:1028B000B7003630C7000A128A1504200A168A119A
:1028C000BA30A200C7000230C80040303E22B23009
:1028D000A200C7000230C80020303E22C630A2004D
:1028E000C7000330C80010303E228430C8000530D5
:1028F000C90083162E088312B600B7013630C70010
:102900000A128A1504200A168A118B178316B4013D
:10291000B50183120317EE010313AF0103176F080C
:1029200003132F020318962CAF0A8E2C2F082D3E6E
:102930008400831780010317ED01EF010230831635
:102940000313A100A601053026020318C62C03308C
:10295000F50026080A168A150F21DB3E8400831332
:1029600080010330F50026080A168A150F210A1681
:102970008A1103138312B800380ADB3E84008313E4
:102980008001840A80018316A60AA32C64008316A2
:10299000201DFA2FD521B001B1018316A508031916
:1029A000FC2CE2308312C8000530C9000A128A15D7
:1029B00004200A168A118316A7080319EB2C33305A
:1029C0008312C8000530C90083162703D13E840056
:1029D00083130008F22C33308312C8000530C9007D
:1029E00083165A088312B600B7013630C7000A12A0
:1029F0008A1504200A168A118312AF012F08D13ECE
:102A0000840083130008B0070318B10AAF0A0A3024
:102A10002F02031CFE2C83162508023A031D1E2DCF
:102A2000F7308312C8000430C9003008B6003108FE
:102A3000B7003630C7000A128A15042083162B0807
:102A4000F4000A128A157A26740803138312B80058
:102A50007508B9007608BA003108F5003008F400AE
:102A60000A128A15FD2783164608F7004708F80062
:102A70004808F9000A128A158027031383123808C0
:102A8000F7003908F8003A08F9000A128A153F27BA
:102A9000F701F8013F30F9000A128A15F1260A12EF
:102AA0008A15C1270A168A117408A3007508A400A4
:102AB0008316A50803196C2DB9308312C8000230A3
:102AC000C9002308B6002408B7003630C7000A1230
:102AD0008A1504200A168A11640083162E0803132F
:102AE0008312B800B90139082402031D792D380872
:102AF0002302031C8D2D8316A5080319892DC830C8
:102B00008312C8000530C9000A128A1504200A166B
:102B10008A118312061586148F2D061186108316CE
:102B20003B083502031D962D3A08340203189B2DED
:102B3000B40A0319B50AA5080319B22D8F30831200
:102B4000C8000430C900831634088312B600831607
:102B500035088312B7003630C7000A128A150420E0
:102B60000A168A1100308316350202300319340226
:102B70000230031CE22D2702031CC42D2703D13E83
:102B8000840083130008C52D5A088312BB00BC01C2
:102B9000831640088312BD00831641088312BE00CD
:102BA000831642088312BF00831634088312C000C4
:102BB000831635088312C1006D210A168A11740824
:102BC0008316F32D2702031CEB2D2703D13E84002F
:102BD00083130008EC2D5A08F4000A128A157A268D
:102BE0000A168A117408C0007508C1007608C20070
:102BF000A5080319312EE6308312C8000330C9003E
:102C0000831640088312B500831641088312B6006C
:102C1000831642088312B7003530C7000A128A159E
:102C200004209130C8000230C90083164608F7001E
:102C30004708F8004808F9004008F4004108F5008A
:102C40004208F6000A128A15802774088312B5001C
:102C50007508B6007608B7003530C7000A128A1525
:102C6000042083164608F7004708F8004808F900D2
:102C70004008F4004108F5004208F6000A128A15DF
:102C800080270A168A117408C3007508C4007608E4
:102C9000C500BB220A168A1183162508023A031DB5
:102CA000652EAC308312C8000430C9008316380882
:102CB0008312B600831639088312B7003630C70076
:102CC0000A128A1504200A168A1103308316270275
:102CD0002708031C842EFE3ED13E84008313000887
:102CE0008312B80083162708FD3ED13E84000008F9
:102CF0008312B90083162703D13E84000008831293
:102D0000390738078316962E023A031D8A2E5A0871
:102D100052078E2E270B902E59085A075107962ED0
:102D2000A708031D972E5A0858075907C9002508F8
:102D3000023A031DAC2EC5308312C8000430C9000E
:102D4000831649088312B600B7013630C7000A124D
:102D50008A1504200A168A118316A6010530260258
:102D60000318002F0330F50026080A168A150F21D4
:102D700003138312B800380ADB3E8400831301304A
:102D80008007840A0318800A0330F500831626089A
:102D90000A168A150F210A168A1103138312B80026
:102DA000380ADB3E840083130008F400840A00081C
:102DB000F5000E307502103003197402031CFD2E4D
:102DC0000330F500831626080A168A150F21DB3E0C
:102DD0008400831380010330F50026080A168A1543
:102DE0000F210A168A1103138312B800380ADB3E3A
:102DF000840083138001840A80018316A60AAE2E04
:102E000067084902031C082F4908E700E801E901A7
:102E10003920640083164608F7004708F800480880
:102E2000F9004008F4004108F5004208F6000A12D3
:102E30008A1580270A168A117408C3007508C40011
:102E40007608C5002508023A031D642FA601053047
:102E500026020318642F75308312C8000430C9009D
:102E60000330F500831626080A168A150F2103136E
:102E70008312B800380ADB3E840083130008F40094
:102E8000840A0008F5007408B6007508B70003301E
:102E9000F500831626080A168A150F21DB3E8400EA
:102EA000831300088312B400B50183162608831229
:102EB000B200B3013230C7000A128A1504200A1684
:102EC0008A118316A60A272F64008312BB01BB0A4E
:102ED000BC01BC0A83164308F7004408F800450803
:102EE000F9000030F401F501F6010A128A15802775
:102EF000F701F8013F30F9000A128A15F1260A128B
:102F00008A15C1270A168A1174088312BD00750834
:102F1000BE00013054228316A20064008312BB015C
:102F2000BC01BC0A83163308F5003208F4000A120B
:102F30008A15FD27F701F030F8004130F9000A1238
:102F40008A153F274308F7004408F8004508F900B0
:102F50000A128A158027F701F8013F30F9000A129A
:102F60008A15F1260A128A15C1270A168A117408D1
:102F70008312BD007508BE00003054228316A200E3
:102F8000A5080319EC2F74308312C8000230C90061
:102F900083165B08F4000A128A157A26F70140307E
:102FA000F800F9000A128A153F274608F70047087B
:102FB000F8004808F9000A128A158027740883125D
:102FC000B5007508B6007608B7003530C7000A129C
:102FD0008A1504200A168A118316A5080319F82FEA
:102FE00014308312C8000630C9000A128A15042062
:102FF000831620110A128A1526210A168A11C72C57
:1030000082074D3461347234203431343634203404
:10301000323430343034383400348207323432348D
:103020003A34343436343A34343432340034FF3FB2
:10320000FF3FFF3FFF3FFF3F830130080A168A154B
:1032100035210A168A152F080A168A153529F40051
:103220000030751874070310F40D0310F50CF50841
:103230000319080011298301E2002E29981C262970
:10324000831698129816831218121816181D2D2915
:103250001A08A100831698129816640083120313AB
:103260000C1E1E296208990008008301B000AF00FF
:10327000B00E0F30B0050A3030020318412930304B
:1032800042293730B00730081B212F08B0000F301B
:10329000B0050A30300203184F293030502937303A
:1032A000B00730081B298301B000AF006430F5007F
:1032B00030080A128A115D270A168A150038643010
:1032C000F50003196D2930080A128A115D270A16C4
:1032D0008A15303E1B216430F50030080A128A112D
:1032E0005D27B1006430F50031080A168A150F21F8
:1032F000B0020A30F50030080A128A115D270A165A
:103300008A1500380A30F5000319902930080A128E
:103310008A115D270A168A15303E1B210A30F500F6
:1033200030080A128A115D27B1000A30F500310811
:103330000A168A150F210A168A15B0023008303E87
:103340001B2983012F08AF003008B0001030F600B1
:103350002730F7003008F5002F08F4000A128A1110
:1033600093270A168A15790878041030F60027305A
:10337000F7000319CB293008F5002F08F4000A12D2
:103380008A1193270A168A157808303E1B211030BF
:10339000F6002730F7003008F5002F08F4000A1275
:1033A0008A1193277808F4007908F5001030F600A8
:1033B0002730F7000A128A151C207808AF02031C78
:1033C000B0037908B002E830F6000330F7003008A7
:1033D000F5002F08F4000A128A1193270A168A159D
:1033E00079087804E830F6000330F7000319082A5A
:1033F0003008F5002F08F4000A128A1193270A16E4
:103400008A157808303E1B21E830F6000330F700BB
:103410003008F5002F08F4000A128A119327780863
:10342000F4007908F500E830F6000330F7000A12DE
:103430008A151C207808AF02031CB0037908B0027B
:103440006430F600F7013008F5002F08F4000A1286
:103450008A1193270A168A15790878046430F600D1
:103460000319412AF7013008F5002F08F4000A1269
:103470008A1193270A168A157808303E1B2164307A
:10348000F600F7013008F5002F08F4000A128A113F
:1034900093277808F4007908F5006430F6000030CE
:1034A000F7010A128A151C207808AF02031CB0032A
:1034B0007908B0020A30F600F7013008F5002F084D
:1034C000F4000A128A1193270A168A1579087804DB
:1034D000031D7A2A6430F600F7013008F5002F0842
:1034E000F4000A128A1193270A168A1579087804BB
:1034F0000319892A0A30F600F7013008F5002F0871
:10350000F4000A128A1193270A168A157808303EA9
:103510001B210A30F600F7013008F5002F08F400EF
:103520000A128A1193277808F4007908F5000A3006
:10353000F6000030F7010A128A151C200A168A15B7
:103540007808AF02031CB0037908B0022F08303EA0
:103550001B29D02A3008EE002F080A128A117E217A
:103560000A168A151B213008EE002F080A128A114C
:103570007E210A168A150D3A031DC02A0A301B2126
:103580003008EE002F080A128A117E210A168A15C9
:103590000A3A031DCD2A0D301B21AF0A0319B00AC8
:1035A000831203133008EE002F080A128A117E21BD
:1035B0000A168A15003803190800AA2A8301D100C7
:1035C000CD014708CB00572E5008253A031D482E41
:1035D000FF30CF00CE01CC01042ED1080319F42A0C
:1035E00051088400831380014D0808000230CB0786
:1035F0004B02840083130008462ECC17042ECC0AFD
:10360000052B0830CF07FE30CF07CC1F172B043017
:10361000CB074B02840083130008F400840A0008DF
:10362000F500840A0008F600840A0008272B0230FF
:10363000CB074B02840083130008F400840A0008BF
:10364000F500740875080030F51BFF30F600F70030
:103650007408DA007508DB007608DC007708DD0006
:103660004C1C512BDD1F602B5A08F4005B08F50041
:103670005C08F6005D08F700F409F509F609F7099A
:10368000F40A0319F50A0319F60A0319F70A74086C
:10369000DA007508DB007608DC007708DD00CE0371
:1036A000612BCC1B602B5B08F5005A08F400F60177
:1036B000F701DA007508DB007608DC007708DD002A
:1036C000CC010B30CF074F08F800F901FA01FB01DC
:1036D0005A08F4005B08F5005C08F6005D08F70086
:1036E0000A128A1198267808D0004F08F800F901CC
:1036F000FA01FB015A30840083130A128A1114273D
:103700000A168A1583120313DE01DE0ADF01E001C7
:10371000E10161085D02031D972B60085C02031D37
:10372000972B5F085B02031D972B5E085A02031C50
:10373000C52B4F08F800F901FA01FB015E30840047
:1037400083130A128A111D260A168A15831203137F
:10375000CE03892BCD0AD1080319BB2B5108840055
:1037600083134C19B52B2030B62B303080008312D8
:103770000313D10AC52B4C19BF2B2030C02B30307E
:103780000A168A151B210A168A15CE034E08803A9E
:103790007F3E0318AA2B4C1CDA2BCD0AD108031943
:1037A000D62B5108840083132D301D2C2D300A1682
:1037B0008A151B214F08F800F901FA01FB015E3060
:1037C000840083130A128A1114270A168A157708AF
:1037D0007604750474040319232C831203135E0802
:1037E000F8005F08F9006008FA006108FB005A0859
:1037F000F4005B08F5005C08F6005D08F7000A12AB
:103800008A1198264F08F800F901FA01FB010A1203
:103810008A1198260A168A157808CE00803A763ED4
:10382000031C142C0730CE07CD0AD1080319202C15
:103830005108840083134E08303E8000D10ADA2BF1
:103840004E08303ED72B0A30831203135002031C5C
:103850002B2C0730D007CD0AD1080319372C51087B
:10386000840083135008303E8000D10A3E2C50085B
:10387000303E0A168A151B210A168A15CC1C572EB3
:10388000CD0AD10803194B2C5108840083132E3024
:103890008000D10A512C2E300A168A151B210A16D7
:1038A0008A155208DA005308DB005408DC0055087A
:1038B000DD000430CC004A08CE004A2D0330CB078F
:1038C0004B02840083130008DE00840A0008DF0036
:1038D000840A0008E00007304F02031C712C0630F8
:1038E000CF004F08CA00CC01F701F801F9015E08CA
:1038F000F4005F08F5006008F6000A128A15202718
:103900000A168A150318982CCC01CC0A5E08F4001C
:103910005F08F5006008F6000A128A1182260A166E
:103920008A157408DE007508DF007608E000CE0313
:10393000CA08031DB62C5E08F7005F08F80060088F
:10394000F900F401F5013F30F6000A128A15F1265C
:103950000A128A15C1270A168A157408DA00750832
:10396000DB007608DC007708DD004A2D4A0ACE022B
:103970005E08F4005F08F5006008F6000A128A1578
:10398000C1277408DA007508DB007608DC007708C8
:10399000DD005A08F4005B08F5005C08F6005D08DD
:1039A000F7000A128A15E9277408F7007508F8006D
:1039B0007608F9005E30840083130A128A15CC263B
:1039C00083120313CC14D601D60AD701D801D9012A
:1039D000F7012030F8004130F9005E308400831395
:1039E0000A128A1577270A30F800F901FA01FB015B
:1039F000831203135630840083130A128A111D2682
:103A00000A168A1583120313CF0BE82CF701F8016D
:103A10003F30F9005E30840083130A128A15CE26E7
:103A2000831203135E08F4005F08F5006008F600D7
:103A30000A128A15C1270A168A157408D200750859
:103A4000D3007608D4007708D50059085502031D25
:103A5000332D58085402031D332D57085302031DFC
:103A6000332D56085202031C4A2D5608D20257081D
:103A7000031C570FD3025808031C580FD4025908CF
:103A8000031C590AD502DA0A0319DB0A0319DC0AF6
:103A90000319DD0A0A30CF00632BCD0AD1080319C0
:103AA000582D51088400831320308000D10A5E2DE8
:103AB00020300A168A151B210A168A15CE034E08D5
:103AC000803A7E3E03184D2D0230CB074B02840016
:103AD00083130008D000482E0230CB074B0284002D
:103AE00083130008DE00840A0008DF00D0015008BC
:103AF0005E07ED005F08EE006D080318EE0A0A127B
:103B00008A117E210A168A1500380319892DD00AD8
:103B1000772D4F08500203188F2D5008CF004F0803
:103B2000CE1BC62DFF3A4E07031CC62DCD0AD10869
:103B30000319A12D51088400831320308000D10A7D
:103B4000A72D20300A168A151B210A168A15CE03C6
:103B50008F2D5F08EE005E080A128A117E210A1678
:103B60008A15D000DE0A0319DF0ACD0AD10803192D
:103B7000C02D51088400831350088000D10AC62D3F
:103B800050080A168A151B210A168A15CF034F0FF3
:103B9000A92D572E4908EE0048080A128A117E21E5
:103BA0000A168A152A3A031DDC2D0230CB074B0278
:103BB000840083130008002E4908EE0048080A120A
:103BC0008A117E21D03ECF00C80A0319C90A4908CC
:103BD000EE0048080A128A117E210A168A15D000C2
:103BE00030305002031C042E3A3050020318042EC9
:103BF0000A30F5004F080A168A150F215007D03EEB
:103C0000CF00C80A0319C90A4908EE004808C80AC3
:103C10000319C90A0A128A117E210A168A15D000D0
:103C2000003A0319ED2A2A3A0319F62A043A03192D
:103C3000CA2D763A0319012B3B3A03195F2D073A37
:103C40000319FF2A023A03195E2C0A3A0319FD2AC6
:103C5000033A0319032B1C3A03196C2D063A031976
:103C6000052B0D3A0319012B30305002031C482E4E
:103C70003A3050020318482E0A30F5004E080A1652
:103C80008A150F210A168A155007D03ECE00042E41
:103C9000CD0AD1080319532E51088400831350080C
:103CA0008000D10A572E50080A168A151B21490890
:103CB000EE004808C80A0319C90A0A128A117E21AF
:103CC0000A168A15D000D008031DE42AD10803196A
:103CD0006D2E51088400831380014D080800FF3FBA
:084000000000000002000000B6
:02400E00351E5D
:00000001FF
